:020000040800F2
:10000000D8190020B1010008B9010008BB0100089F
:10001000BD010008BF010008C10100080000000088
:10002000000000000000000000000000C301000804
:10003000C501000800000000C7010008C901000850
:10004000CB010008CB010008CB010008CB01000860
:10005000CB010008CB010008CB010008CB01000850
:10006000CB010008CB010008CB010008CB01000840
:10007000CB010008CB010008CB010008CB01000830
:10008000CB010008CB010008CB010008CB01000820
:10009000CB010008CB010008CB010008CB01000810
:1000A000CB010008CB010008CB010008CB01000800
:1000B000CB010008310B0008CB010008CB01000880
:1000C000CB010008CB010008CB010008CB010008E0
:1000D000CB010008A10B0008CB010008CB010008F0
:1000E000CB010008CB010008CB010008CB010008C0
:1000F000CB010008CB010008CB010008CB010008B0
:10010000CB010008CB010008CB010008CB0100089F
:10011000CB010008CB010008CB010008CB0100088F
:10012000CB010008CB010008CB010008CB0100087F
:10013000CB010008CB010008CB010008CB0100086F
:10014000CB010008CB010008CB010008CB0100085F
:10015000CB010008CB010008CB010008CB0100084F
:10016000CB010008CB010008CB010008CB0100083F
:10017000CB010008CB010008CB010008CB0100082F
:10018000CB010008CB010008CB010008CB0100081F
:10019000CB010008CB010008DFF810D000F036F8E2
:1001A0000048004769100008AFF30080D81900200C
:1001B0000648804706480047FEE7FEE7FEE7FEE701
:1001C000FEE7FEE7FEE7FEE7FEE7FEE7810A00083E
:1001D0009901000840EA01039B0703D009E008C920
:1001E000121F08C0042AFAD203E011F8013B00F8FC
:1001F000013B521EF9D27047034611F8012B00F85B
:10020000012B002AF9D1184670470000064C074D13
:1002100006E0E06840F0010394E8070098471034D6
:10022000AC42F6D3FFF7BCFF8C100008AC100008FE
:1002300010B504462D480078052855D2DFE800F0B7
:100240000309131D2700552C02D1012027490870EE
:100250004AE0552C03D102202449087002E0002016
:100260002249087040E0012C03D103201F49087087
:1002700002E000201D49087036E0012C03D1042063
:100280001A49087002E00020184908702CE0AA2CD6
:1002900029D172B608221649164800F0C4FC00F0B5
:1002A000E9FB012080F3138800BF00BF00BF00BF3F
:1002B00000BF00BFBFF34F8F00BF00BF00BF0E489D
:1002C000006800F4E0600D490843001D0A49086019
:1002D00000BF00BF00BFBFF34F8F00BF00BF00BF14
:1002E00000BF00BFFDE700BF00BF10BD040000203D
:1002F00010000020003801400CED00E00000FA057D
:1003000008B50121402000F0B9F94FF47850ADF85C
:10031000000004208DF8030003208DF802006946D8
:10032000014800F0E6F808BD0018014070B54FF430
:100330000071154800F068F905014FF4806112481A
:1003400000F062F945EAC0054FF400610E4800F084
:100350005BF945EA80054FF480510B4800F054F9F1
:1003600045EA40054FF40051074800F04DF90543B8
:10037000ECB206480078844204D0204600F04EF9E2
:100380000248047070BD0000001801401C000020ED
:100390000249C9680143014AD16070470020024008
:1003A00030B5044606257C20FFF7F2FF4FF43020DD
:1003B00000F08CF80546062D17D10D48006940F075
:1003C00002000B49086108464461006940F04000A2
:1003D00008614FF4302000F079F8054604480069C0
:1003E00043F6FD71084002490861284630BD00000F
:1003F0000020024006201249C96801F0010109B13C
:1004000001201CE00E49C96801F0040109B1032074
:1004100015E00B49C96801F0080109B104200EE09C
:100420000749C96801F0100109B1052007E0044936
:10043000C96801F0400109B1072000E006207047BB
:10044000002002400348006940F080000149086133
:10045000704700000020024078B504460D4606268D
:100460000020009004F0030010B10926304678BD4A
:100470007C20FFF78DFF4FF4005000F027F8064670
:10048000062E12D10A48006940F0010008490861AF
:1004900025604FF4005000F019F806460448006942
:1004A00043F6FE710840024908613046DFE700006C
:1004B00000200240024803494860034848607047F2
:1004C0002301674500200240AB89EFCD00B502460D
:1004D0000623FFF78FFF034603E0FFF78BFF03467A
:1004E000521E012B01D1002AF7D102B90A23184666
:1004F00000BD2DE9F0410246002500260020002322
:100500000024002791F803C00CF00F0591F803C0F8
:100510000CF0100CBCF1000F03D091F802C04CEAB3
:10052000050591F800C0BCF1000F31D0146800201F
:100530002BE04FF0010C0CFA00F3B1F800C00CEA0C
:1005400003069E4220D183004FF00F0C0CFA03F7F4
:10055000BC4305FA03FC4CEA040491F803C0BCF167
:10056000280F06D14FF0010C0CFA00FCC2F814C0A1
:100570000AE091F803C0BCF1480F05D14FF0010C1F
:100580000CFA00FCC2F810C0401C0828D1D314603B
:10059000B1F800C0BCF1FF0F34DD546800202EE03C
:1005A00000F1080C4FF0010808FA0CF3B1F800C094
:1005B0000CEA03069E4221D183004FF00F0C0CFA87
:1005C00003F7BC4305FA03FC4CEA040491F803C0AA
:1005D000BCF1280F05D100F1080C08FA0CF8C2F89C
:1005E000148091F803C0BCF1480F07D100F1080C4A
:1005F0004FF0010808FA0CF8C2F81080401C0828D7
:10060000CED35460BDE8F0810246002093680B40D1
:100610000BB1012000E00020704700003EB5044609
:1006200007250AE004F0010008B1312200E0302281
:1006300028466D1E0DF800206410002CF2DC04E04A
:10064000302228466D1E0DF80020002DF8DA00201B
:100650008DF808006A4602A100F086F83EBD000051
:1006600044697020537769746368204164647265DB
:1006700073733A2025730D0A0000000029B1064A61
:1006800092690243044B9A6104E0034A92698243EF
:10069000014B9A6170470000001002402DE9F041C3
:1006A00004460D4616460E4F00BF387808B900F0D4
:1006B000F9FA00BFEFF311800746202080F311887C
:1006C00000BF00BF32462946204600F00BF88046A6
:1006D000F8B280F3118800BF00BF4046BDE8F0814A
:1006E000200000202DE9F047074688461646C246FE
:1006F00007EB47011B4800EBC109D9F8140020B1F2
:10070000012811D0022826D11EE0484600F002FB45
:100710000546B54201D2002405E034463246514632
:10072000484600F04EFC18E0484600F0F3FA054653
:10073000B54201D2284600E03046044622465146E2
:10074000484600F03EFC08E032465146484600F07C
:10075000FDFB044601E0002400BF00BF2046BDE8C9
:10076000F0870000380000200FB438B5044606A812
:1007700000906A462046059900F007F805460020DB
:100780000090284638BC5DF814FB2DE9F04F99B075
:1007900082460D46144603A8149040201590002070
:1007A0001690CDF860A0179000BF2E786D1C06B98A
:1007B000DDE0252E79D100274FF0010900BF2E780A
:1007C000232E12D02B2E0CD02D2E02D0302E10D155
:1007D00003E047F001076D1C0EE047F002076D1CB7
:1007E0000AE047F004076D1C06E047F008076D1C9F
:1007F00002E04FF0000900BF00BFB9F1000FDED1E9
:100800004FF0000800BF2E78302E01DB392E00DDBE
:1008100007E06D1CA6F1300008EB880100EB4108F1
:10082000F1E700BF002013902E782E2E12D16D1C00
:1008300000BF2E78302E01DB392E00DD09E06D1C63
:10084000A6F13000139901EB810100EB41001390F8
:10085000EFE700BF2E7800BF6C2E01D0682E02D1CA
:100860006D1C2E7800E000E0F6E700BF702E5DD032
:1008700008DC252E6AD0582E35D0632E09D0642E80
:1008800069D113E0732E3CD0752E1DD0782E62D125
:1008900028E02168081D2060D1F8009009F0FF0BC6
:1008A000594614A800F030FB56E058E02168081DB6
:1008B0002060D1F80090CDE900870A22494614A8AB
:1008C000139B00F035FA47E02168081D2060D1F83D
:1008D0000090CDE900870A22494614A8139B00F036
:1008E0009DFA39E000BF2168081D2060D1F8009012
:1008F000CDE900871022494614A8139B00F08EFA18
:100900002AE02168081D2060D1F800B000BF9BF8E4
:1009100000600BF1010B06B906E0314614A800F0A7
:10092000F3FA17980028F2DA00BF15E02168081DD5
:100930002060D1F80090002008210B461022CDE95C
:100940000010494614A800F069FA05E0252114A812
:1009500000F0DAFA00E000BF00BF6D1C03E0314692
:1009600014A800F0D1FA17980028BFF61EAF00BFF8
:10097000179800280ADD169820B103A95046169A48
:10098000FFF78CFEDDE9161008441790179819B090
:10099000BDE8F08F10B50020002100222F4B1B680E
:1009A00043F480332D4C236000BF2C4B1B68C3F3F2
:1009B0004041521C11B9B2F5004FF6D1274B1B68CC
:1009C000C3F3404119B9264B264C236010BD264B7A
:1009D0001B6823F00303244C236023461B6843F069
:1009E000040323601D4B5B681C4C636023465B68FB
:1009F00043F40053636023465B6843F4A063636081
:100A000023465B68194C2340144C636023465868A6
:100A100040F4803000BF164B1843234658601B68D3
:100A200043F08073236000BF0C4B1B6803F000731E
:100A3000002BF9D0094B5B6823F00303074C63607C
:100A400023465B6843F00203636000BF034B5B68AF
:100A500003F00C03082BF9D100BFB7E700100240E8
:100A600000127A000000002000200240FFFFC0F7C3
:100A70000000040810B54FF0553000F0FBF810BD31
:100A800010B52448006840F47000224908602248EC
:100A9000006840F0010020490860084640681F498E
:100AA00008401D494860084600681D4908401A4929
:100AB00008600846006820F4802008600846406806
:100AC00018490840144948600020C86208634FF480
:100AD0001F0088600846C06940F08050C861124815
:100AE000C06840F001001049C8600B48C06920F0A0
:100AF00080500949C8610D48006840F090000B49DA
:100B00000860FFF747FF4FF0006002498039086036
:100B100010BD000088ED00E00010024000C0FFF8AA
:100B2000FFFFF6FEFFFF00F70070004000200240CC
:100B300010B501210B4800F021F888B101210948C6
:100B400000F018F808480068401C0749086008468B
:100B5000006806490968884202D9002004490870E3
:100B600010BD000000040040180000200800002014
:100B70000400002002698A430261704730B50246D2
:100B8000002000230024156905EA0103958905EA80
:100B9000010413B10CB1012000E0002030BD0000C1
:100BA00010B540F225510A4800F027F878B140F21C
:100BB0002551074800F012F8054800F02BF8C4B2A0
:100BC00004480068044908602046FFF731FB10BD67
:100BD00000380140180000200800002010B5002255
:100BE000002340F66A14A14200D100BF0A1201247A
:100BF0009440A3B2DC43048010BD02460020B1F54E
:100C0000007F00D100BF13880B400BB1012000E032
:100C10000020704701468888C0F308007047C1F380
:100C20000802828070472DE9F04107460D461646BE
:100C3000002405E0295D384600F00DF8601CC4B2C0
:100C4000B442F7DB00BF40213846FFF7D6FF00284B
:100C5000F9D0BDE8F08170B504460D46294620461E
:100C6000FFF7DDFF00BF80212046FFF7C6FF002809
:100C7000F9D070BD10B50446FFF71CFC0848FFF71B
:100C80008FFB21460648FFF7E7FB062803D0FFF756
:100C9000D9FB012010BDFFF7D5FB0020FAE70000CB
:100CA00000FC070810B5124C03202061606111A000
:100CB000A0611349E1614FF4806121620021A162CA
:100CC0006162E1620BA020660E4961661021A16697
:100CD00000212167E16661670BA1E01DFFF78CFA37
:100CE0000AA12046FFF788FA2020A07110BD00005D
:100CF000200000205465726D696E616C0000000078
:100D0000C8000020C80400205254540053454747EF
:100D10004552000010B501460A69CB689A4204D8D2
:100D20008C68641EE41AA01801E0D41A601E10BD7D
:100D30002DE9FC5F06460F4692469846DDE90C45D4
:100D4000002F01DA784200E0384683464FF001096F
:100D500003E09BFBFAFB09F10109D345F9DAC84529
:100D600000D9C14634B1002F03DB05F0040004288C
:100D700000D1641E05F0020010B1B8F1000F11D0CF
:100D800005F0010070B96CB108E0641E2021304606
:100D900000F0BAF8F068002800DA02E00CB1A145D2
:100DA000F3D300BFF068002836DB002F05DA7F425E
:100DB0002D21304600F0A8F807E005F004000428D3
:100DC00003D12B21304600F09FF8F068002823DB88
:100DD00005F00200022814D105F0010088B9B8F12D
:100DE000000F0ED16CB108E0641E3021304600F0D7
:100DF0008BF8F068002800DA02E00CB1A145F3D3CB
:100E000000BFF068002807DB4346524639463046AB
:100E1000CDE9004500F002F8BDE8FC9F2DE9FC5F3C
:100E20008046894615461E460C9CCDF80490012745
:100E3000BB4605E00198B0FBF5F001900BF1010B0A
:100E40000198A842F6D25E4500D9B3460D9800F04D
:100E50000100D0B9CCB10D9800F00200022803D1F6
:100E600016B93020009001E02020009009E0641EB7
:100E70004046009900F048F8D8F80C00002800DA45
:100E800002E00CB1A345F2D300BFD8F80C00002853
:100E900035DB09E0012E01D9761E04E0B9FBF7FA33
:100EA000AA4500D201E06F43F4E700BF00BFB9FBE1
:100EB000F7FA0AFB1799134810F80A10404600F099
:100EC00023F8D8F80C00002800DA03E0B7FBF5F7A8
:100ED000002FECD100BF0D9800F0010078B174B183
:100EE00009E0641E2021404600F00EF8D8F80C00FE
:100EF000002800DA02E00CB1A345F2D300BFBDE840
:100F0000FC9F00007C10000870B504460E46A568E2
:100F1000681C6168814206D320684655681CA06041
:100F2000E068401CE060D4E9011088420DD1A2685D
:100F300021682069FFF7B2FBA168884203D04FF017
:100F4000FF30E06001E00020A06070BD2DE9F05F9F
:100F50000446894617464FF0000AE56800BFD4F8FA
:100F60001080A84503D9A8EB0500461E04E0A5EBB8
:100F70000800401CA1680E1AA068401BB04201D9AD
:100F8000304601E0A068401B0646BE4201D2304612
:100F900000E038460646606800EB050B32464946DD
:100FA0005846FFF717F9B244B144BF1B3544A06857
:100FB000A84200D10025E560002FD0D15046BDE801
:100FC000F09F2DE9F047044689461546E668A0687B
:100FD000871BAF420AD9606800EB060A2A464946D9
:100FE0005046FFF7F7F87019E06014E0B846606803
:100FF00000EB060A424649465046FFF7EBF8A5EBE0
:101000000708D4F804A009EB070142465046FFF751
:10101000E1F8C4F80C80BDE8F08702E008C8121FB0
:1010200008C1002AFAD170477047002001E001C1D1
:10103000121F002AFBD1704710B5002100220023A7
:1010400000BF00BF00BF00BF0BE00023002203E091
:101050005C1CA3B2541CA2B2B2F5165FF8DB4C1CA8
:10106000A1B28142F1DB10BDFFF74AF905E0FFF7BD
:101070005DF94FF47A70FFF7DFFFF8E73031323374
:10108000343536373839414243444546AC100008C0
:1010900000000020200000001A100008CC100008FA
:1010A00020000020B81900002A100008004495080C
:1010B0000000000000000000000000006666666698
:0C10C0006666666600000000000000008C
:04000005080001B13D
:00000001FF
